:020000040000FA
:0200000057D0D7
:040008009EEF19F05E
:08001800F0EF19F00F0B7C6EF4
:10002000000EF76E360EF66E7C50F626D8B0F72A24
:100030000800F55012003031323334353637383954
:100040004142434445460F501F0B7C6E000EF76E35
:10005000540EE9D72C36404A545E68727C86909ADA
:10006000A4AEBECEDEEE070B7C6E000EF76E720EF7
:10007000DAD70A0E12161A1E59507C6ED8907C32AE
:100080007C327C301F0B7C6E000EF76E900ECBD74F
:1000900085786D645C56504B47433F3C393734326A
:1000A000302E2C2B292827262423222120201F1EF6
:1000B00029DB828AF8EC17F061DA2E8C72682D80C9
:1000C000010E526E100E8F6FFF0E056E27EC0CF0B6
:1000D0000650650810E121DA28E361DB010E365C89
:1000E00006E1D1EC0BF047DB56DB07EF17F057DBEF
:1000F000040E365C16E1DFDA000EF86E380EF76E8D
:100100008C0EF66E73EC03F0FFEC0BF0D4DA000EFD
:10011000F86E380EF76E9E0EF66E73EC03F00ADA88
:1001200023DAFBD9FEE258EF00F0000EF86E380E2D
:10013000F76E080EF66E73EC03F05A6A056A27EC48
:100140000CF012EC0CF0052A5A2EF9D79CEC02F0B8
:10015000D1EC0BF010DB0CDA0FC030F090EC0BF0B0
:1001600010BC04D019EC09F03AEC09F08EEC19F04F
:1001700096EC19F08EEC19F096EC19F03DEC0CF0C1
:1001800010B4838410B28384010E0E6E10A603D0C7
:100190002CB001D00E6AFFDA726883B202D083B04D
:1001A00096D92E8837523CE010B483842E98F3DA27
:1001B00037502DA21ED037BE0BD07C0B31E0522A17
:1001C000050E10BC0D0E525C02E1010E526E0DD0F8
:1001D00037C05DF05D6C5D50FC0B22E0520652288A
:1001E00004E1040E10BC0C0E526E2E8C7268376A3D
:1001F00017D037BE09D0376A7F0B5D6E2EAA6EEC22
:1002000005F05D2EFBD709D0376C3750376A5D6E2D
:100210002EAAADEC05F05D2EFBD72E8C72682D80DA
:100220002EAC19EF01F02E9872EC07F043EC07F0BA
:100230002E9C2DA004D02E98C9DA2BDB2D906DD9E1
:100240002DAC20D010B483842E98A5DA2DA405D02F
:100250002D948DEC02F0FDE215D0A1DA010E365C92
:1002600002E114EC0AF0020E365C02E122EC0AF024
:10027000030E365C02E15DEC0AF0040E365C02E12E
:1002800098EC0AF02FA003D02E982E8C72682F9A2B
:10029000010E315C05E0020E315C02E02F8A1ED0B7
:1002A00010A81CD081B408D02DA205D02D8436EC26
:1002B00018F02D9401D02E8281A22E842EA21CD063
:1002C0002E98E9DA83802D8483827CEC02F083927D
:1002D000F7D82D947CEC02F02E92F1D081B40AD0A4
:1002E00083B206D02E98D7DA838083822FAA2D84FA
:1002F000E7D8E5D083922D94010E315C03E0020E25
:10030000315C17E110A815D02EA413D02E98C3DAB3
:1003100083802D8483827CEC02F07CEC02F07CEC08
:1003200002F08392CDD8D3D82D947CEC02F02E9499
:10033000C6D0535209E02DAE12D010B283842D9E48
:100340002E802E8C72680AD02EA009D010B483940F
:1003500010B283842F902E902E8C72682E982CA031
:100360001DD057661BD0030E0E6E100ED06102D04A
:10037000020E0E6E0A0ED06102D0010E0E6E040E39
:10038000D06102D0000E0E6ED151D05D04E0D0C01D
:10039000D1F02E8C7268D06B0A0E576E2EA88FD0BB
:1003A000010E8F5D27E110AC19EC09F00F50305CA5
:1003B00021E010ACDDD87FD930508ED9000EF86E18
:1003C000380EF76E580EF66E73EC03F0AAEC0BF0D5
:1003D00030C00FF090EC0BF0ADD82E8C72682D80F1
:1003E000DAD910B483842CB002D0010E0E6E10BC8A
:1003F0008EEC19F0020E8F5D1AE110AC3AEC09F0A8
:100400000F5201E1326A3250315C11E032C031F0FA
:100410002EA604D031C025F031C026F069EC0BF0D7
:10042000BAD910B483842D8010BC96EC19F0030E59
:100430008F5D08E110A006D047EC08F06F50725CA9
:1004400001E02E8C040E8F5D23E110A821D07736B9
:10045000783677367836773678367736783678C0A5
:1004600075F05850785E10E075C078F05828785EC6
:100470000BE075C078F05804785E06E010B4838411
:100480002F8089D975C058F0756A766A776A786A5C
:10049000050E8F5D02E109EC18F0060E8F5D00E19C
:1004A00010A809D05BEC09F08EC075F0766A755023
:1004B0007726765078228F2F02D0100E8F6F6DD650
:1004C000000ECE6EA60ECF6E12C054F01200010EBA
:1004D000315C04E0020E315C01E001D02D945452F5
:1004E00002E18390D6D912009EAAFED7AE50120028
:1004F0009EA8FED7AD6E12005BEC09F0BDDD566E16
:10050000F20ECB6ECA8481A42E8281A22E8483A295
:10051000DEDF5652F8E1CA9412002D9C8150F00B98
:10052000F00A03E02D8CD88001D0D890120001D8B9
:1005300001D800D802D801D800D8FA0E09D0C80EC8
:1005400007D0640E05D0320E03D00A0E01D0010E82
:10055000356E070E346E7D0E336E332EFED7342E7D
:10056000FCD7352EF6D712002D84EDDF2D94EBDF6E
:100570002D84E9DF2D9483908392120083968296D6
:100580008298E1DF200E78D8800E76D8DEDF200E4C
:1005900073D8800E71D8DBDF060E64D80C0E62D8DB
:1005A000140E60D830D887D8000EF86E390EF76E6A
:1005B000A80EF66E73EC03F0000EF86E330EF76EB5
:1005C000F60EF66E73EC03F0B4DF75D88384120078
:1005D000076E5ED80750828682988396F00B4CD8BF
:1005E0000738F00B49D0076E07460746074650D834
:1005F0000750400937D8080E5A6E0900F550E8DF59
:100600005A2EFBD71200000EF86E060EF76E240E5F
:10061000F66E080E5B6E5C6A5C50E5DF5C2A5B2E52
:10062000FBD7120000001818181B000000001B1B4D
:100630001B1B000004041818181B040404041B1BD3
:100640001B1B0404001010101010100000141414D0
:100650001414140000000000001B00000404040433
:10066000041B0404076E14D80750F00B829682987E
:10067000839602D80738F00B83B0010983B20209D0
:1006800083B4040983B60809836E838683961200B7
:10069000838E958E829682882D968386000083AE07
:1006A0002D86839600008386000083962DA6F4D7BE
:1006B000959E82981200010ED5D7020ED3D7800ED8
:1006C000D1D7C00ECFD78009CDD7200E81D75A6E93
:1006D000FCDF5A2EFDD71200086E08389FDC78DF49
:1006E00008509CDC75D70900F550EDDF0900F55086
:1006F00002E06EDFFBD712000900F55002E0F8DEE1
:10070000FBD71200800EC16E2F0E926EFF0E936EFD
:10071000800E946E000E956E070E966E000ED06ED3
:10072000F00EF26E000EF16E000EF06E230E9D6E56
:10073000020EA06E010ECD6E210ECA6E000EB16EBD
:100740002F0E806EFF0E816E000E826E000E836E85
:10075000070E846EFF0E5A6E00EE00F0EE6A5A2EFF
:10076000FDD710B4838410B28384000ECE6EA60E23
:10077000CF6ECBEF03F091D81C0E436E200E426E6D
:10078000BFC04AF0A7DA77DA38C066F0660ED66ED8
:10079000C40ED56E1200C80E536E2D8E1200280E98
:1007A0005A6E8150F00B5B6ED2DE8150F00B5B5CB9
:1007B000F6E15A2EF6D7000E5BAE010E5BAC020ED0
:1007C0005BAA030E5BA8040E366E120066D89CD896
:1007D00010EE42F0050E5A6EEE50E66E5A2EFCD721
:1007E0000F5207E010A619EC05F02FA201D910BE98
:1007F00044D809C04AF00AC04BF00BC04CF00CC002
:100800004DF00DC04EF0FDD93CC05EF03DC05FF034
:100810003EC060F03FC061F040D87CD810EE42F09E
:10082000050E5A6EEE50E66E5A2EFCD70F5211E0AE
:1008300010A619EC05F02FB20AD0010E315C05E0CC
:10084000020E315C02E094D802D010BA91D810BEEA
:1008500014D809C04AF00AC04BF00BC04CF00CC0D1
:100860004DF00DC04EF0CDD93CC062F03DC063F0FC
:100870003EC064F03FC065F01200D8904236433667
:100880004436453646364236433644364536463695
:100890001200A6EF0CF0B8EF0CF013D809D8426A9A
:1008A000436A446A456A466A476A486A496A120066
:1008B0004A6A4B6A4C6A4D6A4E6A4F6A506A516A7C
:1008C0001200386A396A3A6A3B6A3C6A3D6A3E6A93
:1008D0003F6A406A416A120038C042F039C043F0B2
:1008E0003AC044F03BC045F03CC046F0120038C06E
:1008F0004AF039C04BF03AC04CF03BC04DF03CC020
:100900004EF0120010EE38F000EE1BF02DB800EEA5
:1009100020F012002EA6F8D700EE1BF02DA800EE56
:1009200020F01200D0D8EECF38F0EECF39F0EECF75
:100930003AF0EECF3BF0200E5B6ED8903B323A326D
:10094000393238323F323E323D323C3200EE38F0FE
:10095000040E5A6EEFAE02D0300EEF5EEFA602D05C
:10096000030EEF5EEE525A2EF5D75B2EE6D712003D
:100970002FB409D017504226185043221950442250
:100980001A50452208D01750425E1850435A195049
:10099000445A1A50455A386A396A3A6A3B6A050E0F
:1009A000315C07E1C00E386E270E396E090E3A6EC3
:1009B00009D0060E315C0EE1800E386EF70E396EEE
:1009C000730E3A6E3850425E3950435A3A50445A88
:1009D0003B50455A45AE1200421E431E441E451E62
:1009E000422AD8B4432AD8B4442AD8B4452A12009B
:1009F0002FB409D0135042261450432215504422DC
:100A00001650452208D01350425E1450435A1550D8
:100A1000445A1650455A45AE1200421E431E441E0B
:100A2000451E422AD8B4432AD8B4442AD8B4452A09
:100A30001200466A58EC04F00A0E4A6E6AEC06F0A0
:100A40006CEC04F058EC04F00A0E4A6E01EC06F06F
:100A50006CEF04F009C042F00AC043F00BC044F050
:100A60000CC045F00DC046F0200E5B6E00EE42F06B
:100A700010EE4AF0396AD8903F323E323D323C3275
:100A8000D8A015D0080E5A6E00EE42F010EE4AF0D3
:100A9000EECF38F03950396AE72602E3010E396E9D
:100AA0003850E62602E3010E396E5A2EF1D7D8905F
:100AB000423643364436453646364736483649365A
:100AC0005B2ED4D71200416A406A3F6A3E6A3D6A93
:100AD0003C6A3B6A3A6A396A386A1200F9DF12DF07
:100AE0002CB00FD00E5031E0010E0E5C2BE0020E48
:100AF0000E5C25E0030E0E5C1AE0040E0E5C10E0A6
:100B000012000E5027E0010E0E5C1CE0020E0E5C7F
:100B100016E0030E0E5C10E0040E0E5C01E0120005
:100B2000A00E386E860E396E010E3A6E61D0030E3D
:100B3000396EE80E386E5CD0C80E386E59D0320E61
:100B4000386E56D00A0E386E53D0382A51D0020E65
:100B5000386E4ED0050E386E4BD0BADFD3DE2CB0D7
:100B60000FD00E5037E0010E0E5C2BE0020E0E5C33
:100B700025E0030E0E5C1AE0040E0E5C10E012007D
:100B80000E5022E0010E0E5C1CE0020E0E5C16E020
:100B9000030E0E5C10E0040E0E5C01E01200A00ECD
:100BA000386E860E396E010E3A6E16D0030E396E0F
:100BB000E80E386E11D0C80E386E0ED0320E386E78
:100BC0000BD00A0E386E08D0050E386E05D0020E16
:100BD000386E02D0382A00D0050E5A6ED86AE75017
:100BE000D8A0E73CEF5EEE52E6525A2EF8D712003C
:100BF000E650EE26040E5A6EE650EE225A2EFCD730
:100C000012000A0E5A6E00EE38F0EE6A5A2EFDD728
:100C10002F9646BE40D84EBE4DD8050E5A6E00EEF9
:100C20004AF020EE38F0050E5B6E5A505B5E10EE17
:100C300042F020EE38F05B5203E0DE525B2EFDD72F
:100C4000050E5B6E030E5C6EEF50E602F350DE267F
:100C5000F450DE22E86ADE225C2EFCD7040E5C6EC5
:100C6000DD525C2EFDD75B2EEDD7EE525A2EDBD730
:100C70002FB601D81200381E391E3A1E3B1E3C1EEC
:100C8000382AD8B4392AD8B43A2AD8B43B2AD8B4A6
:100C90003C2A2F961200421E431E441E451E461E2D
:100CA000422AD8B4432AD8B4442AD8B4452AD8B45E
:100CB000462A0ED04A1E4B1E4C1E4D1E4E1E4A2A60
:100CC000D8B44B2AD8B44C2AD8B44D2AD8B44E2A1A
:100CD0002F7612002F9646BEDEDF4EBEEBDF4E9E15
:100CE000469E5A6AEEDD5A2AD8904EBE1BD04A362E
:100CF0004B364C364D364E364E50465C0BE14D5021
:100D0000455C08E14C50445C05E14B50435C02E11A
:100D10004A50425CE8E2D5DDD8904E324D324C323A
:100D20004B324A324E50465C0BE14D50455C08E177
:100D30004C50445C05E14B50435C02E14A50425C3C
:100D40000AE34A50425E4B50435A4C50445A4D506D
:100D5000455A4E50465A383639363A363B363C3686
:100D60005A2EDAD72FB687DF1200386A396A3A6A04
:100D70003B6A3C6A3D6A280E5A6E060E5B6E00EEB8
:100D800038F0EF500F0B7D6E050E7D5CD8A002D0C1
:100D9000030EEF26EF50F00B7D6E500E7D5CD8A059
:100DA00002D0300EEF26EC525B2EEBD7D8904236B5
:100DB0004336443645364636383639363A363B368B
:100DC0003C363D365A2ED9D712002F9C8CBF2F8C23
:100DD0008C9F00EE7EF00C0E5A6E8A515A5C8A6F20
:100DE0008B515A5C8B6F2D9A8C515A5E8B07D8B4FD
:100DF0002D8A8B2B8B5303E12C0EE8EC02F0EE5086
:100E00005B6E8A530CE12DBA06D0300E5B5C03E1B9
:100E1000200E5B6E01D02D8A5B50E8EC02F08A5305
:100E200001E08A078B075A2EE1D78C5303E08C51DF
:100E30002FAC4DDC12007E6A7F6A806B816B826B07
:100E4000836B846B856B866B876B886B896B00EE1D
:100E50007EF010EE3DF0060E5A6EE7380F0B05D807
:100E6000E55003D85A2EF9D712000F0B3009EE6E59
:100E700012000F0B04E12DAA02D0200E02D030097F
:100E80002D9AE8EF02F02DB24AD22FB0CCD00F52FB
:100E900002E010B044D1400E16DC410E2DA8420EE7
:100EA0002EA603D0610E2DA8620EE8EC02F02DB83C
:100EB0000BD020C042F021C043F022C044F023C038
:100EC00045F024C046F00AD01BC042F01CC043F0DD
:100ED0001DC044F01EC045F01FC046F032D8030EBE
:100EE00067EF03F0E86A63EC03F0410E2DB8420EA1
:100EF0002EA603D0610E2DB8620EE8EC02F02DB8DC
:100F00000BD01BC042F01CC043F01DC044F01EC0FB
:100F100045F01FC046F00AD020C042F021C043F087
:100F200022C044F023C045F024C046F00AD82CA0CB
:100F300006D00C0E63EC03F02E0EE8EC02F0BAEFD4
:100F400007F000EE42F010EE27F052DE0EDF73DF06
:100F50000B0E8A6F060E8B6F010E8C6F2CB007D0B4
:100F60000EC08CF0040E0E5C02E1050E8C6FE5ECF9
:100F700006F012000D0E63EC03F010BE02D03152E9
:100F800009E1000EF86E380EF76E2E0EF66E73EC59
:100F900003F01200010E315C09E1000EF86E380E0C
:100FA000F76E340EF66E73EC03F01200020E315C35
:100FB00009E1000EF86E380EF76E3A0EF66E73EC1D
:100FC00003F01200030E315C09E1000EF86E380EDA
:100FD000F76E400EF66E73EC03F01200040E315CF7
:100FE00009E1000EF86E380EF76E460EF66E73ECE1
:100FF00003F01200050E315C09E1000EF86E380EA8
:10100000F76E4C0EF66E73EC03F01200060E315CB8
:1010100009E1000EF86E380EF76E520EF66E73ECA4
:1010200003F0120012000F52D8B41200000EF86E36
:10103000380EF76E720EF66E73EC03F05BEC09F08F
:101040005D6E5D325D325D301F0B090F5D6E25DC1C
:101050005DC042F08ADE38506CEC03F0090E67EF99
:1010600003F0B7C04AF0B8C04BF0B9C04CF0BAC0FA
:101070004DF0BABF4E681200BBC04AF0BCC04BF086
:10108000BDC04CF0BEC04DF0BEBF4E6812004DEC6E
:1010900004F06AEC09F08DC042F08EC043F031ECF0
:1010A00008F001EC06F06CEC04F03CEC08F04A505F
:1010B00042264B5043224C5044224D5045224E5024
:1010C000462246BE4FEC04F058EC04F0500E4A6E37
:1010D000C30E4B6E000E4C6E4A5042264B504322BC
:1010E0004C5044224D5045224E50462258EC04F0BC
:1010F000A00E4A6E860E4B6E010E4C6E6AEC06F028
:1011000038C06FF038C071F0712AD890713242C087
:1011100070F06FAE03D06F6A706A716A120072501D
:101120006F5CD8B448D06FC072F0400E63EC03F02F
:101130000D0E5A6E050E5A6202D0070E01D0060E31
:10114000E8EC02F05A2EF6D7400E63EC03F06FC0C5
:101150005AF0D8905A325B6A5A520EE05B2A0E0E51
:101160005B6018D0090E5B6202D0030E01D0010E45
:10117000E8EC02F05A2EF2D76FA00CD05B2A0E0ECC
:101180005B6008D0090E5B6202D0020E01D0000E37
:10119000E8EC02F04E0E63EC03F0530EE8EC02F0C4
:1011A000090E716404D02B0EE8EC02F004D07150EB
:1011B0003009E8EC02F012006F506CEC03F065ECC3
:1011C00003F070506CEC03F065EC03F071506CECC4
:1011D00003F065EC03F012004DEC04F05BEC03F05F
:1011E00085D8C3CF4AF0C4CF4BF0260E436E4D0EC8
:1011F000426E01EC06F0426A436A446A456A466AF6
:101200003AC042F039BE422AB0DD15DE030E8A6FC5
:10121000010E8B6F8C6B030E63EC03F0D6DD000EBA
:10122000F86E380EF76E6A0EF66E73EC03F099EFF7
:1012300002F04DEC04F050D8C3CF42F0C4CF43F0DD
:101240001E0E4A6E000E4B6E4A5042264B504322F1
:101250004A6A4B6A4C6A4D6A4E6A640E4A6ED1DC29
:101260006CEC04F0170E4B6E810E4A6E33DD38C005
:1012700030F012004DEC04F02BD8C3CF42F0C4CFB5
:1012800043F0660E4A6E000E4B6E4A5042264B509B
:1012900043224A6A4B6A4C6A4D6A4E6A640E4A6E31
:1012A000B0DC6CEC04F04F0E4B6EEC0E4A6E12DDAF
:1012B0003828326E1200C19E17D88E51596EC18ED9
:1012C000120014D8C3CF67F0C4CF68F02E8E12007E
:1012D000F90E0DD0F10E0BD0E90E09D0E10E07D0BA
:1012E000D90E05D0D10E03D0C90E01D0C10EC26EE9
:1012F000640E5A6E5A2EFED7C284C2B4FED7C4CF33
:101300008EF0C3CF8DF01200386E6E0E3802F3CF20
:1013100038F0F4CF39F038BE392A39501200010EB6
:10132000525C08E1000EF86E380EF76ED00EF66EC5
:1013300073EC03F0020E525C08E1000EF86E380EFA
:10134000F76EE20EF66E73EC03F0030E525C08E1EA
:10135000000EF86E380EF76EF40EF66E73EC03F0B6
:10136000040E525C08E1000EF86E390EF76E060EA0
:10137000F66E73EC03F0050E525C08E1000EF86E99
:10138000390EF76E180EF66E73EC03F0060E525C13
:1013900008E1000EF86E390EF76E2A0EF66E73EC49
:1013A00003F0070E525C08E1000EF86E390EF76E7E
:1013B0003C0EF66E73EC03F0080E525C08E1000E72
:1013C000F86E390EF76E4E0EF66E73EC03F0090EE2
:1013D000525C08E1000EF86E390EF76E600EF66E84
:1013E00073EC03F00A0E525C08E1000EF86E390E41
:1013F000F76E720EF66E73EC03F00B0E525C08E1A2
:10140000000EF86E390EF76E840EF66E73EC03F074
:101410000C0E525C08E1000EF86E390EF76E960E57
:10142000F66E73EC03F012002E9A376AB8EC02F0F5
:101430002D722DB202D0010E526E2E8C72685BECB2
:1014400003F0C0D022D9010E525C01E117D9020E7F
:10145000525C01E1EED8030E525C01E1DFD8040ECC
:10146000525C02E136EC18F0050E525C02E1010E0E
:10147000326E060E525C02E1020E326E070E525CB4
:1014800002E1000E306E080E525C02E1030E306E77
:10149000090E525C02E1060E306E0A0E525C02E149
:1014A000090E306E0B0E525C02E10C0E306E0C0E0B
:1014B000525C02E10F0E306E81D0E7D8010E525C13
:1014C00001E1C9D8020E525C01E1BED8030E525CA4
:1014D00002E140D97CD9040E525C01E1A9DA050E83
:1014E000525C02E1030E326E060E525C02E1050E02
:1014F000326E070E525C02E1010E306E080E525C35
:1015000002E1040E306E090E525C02E1070E306EED
:101510000A0E525C02E10A0E306E0B0E525C02E1C2
:101520000D0E306E0C0E525C02E1100E306E46D085
:10153000ACD8010E525C01E14DD8020E525C09E1BB
:10154000040E0E5C05E0040E0E6E2E8C726801D047
:1015500082D8030E525C05E12C70F9EC0BF0010E01
:101560000E6E040E525C02E137DE14D1050E525CA1
:1015700002E1040E326E060E525C02E1060E326E7D
:10158000070E525C02E1020E306E080E525C02E160
:10159000050E306E090E525C02E1080E306E0A0E26
:1015A000525C02E10B0E306E0B0E525C02E10E0E2D
:1015B000306E0C0E525C02E1110E306E366A010E76
:1015C000526E2D928DEC02F0FDE25BEC03F02E8C5E
:1015D000726812002EB60BD016D82DB804D01ED8C3
:1015E00025C026F006D025D826C025F002D006D882
:1015F00038D92E762E8C72682D80120010EE1BF0DA
:1016000020EEABF004D020EE1BF010EEABF00C0E91
:101610005A6EDECFE6FF5A2EFCD712001BC020F018
:101620001CC021F01DC022F01EC023F01FC024F0FA
:10163000B1D020C01BF021C01CF022C01DF023C07F
:101640001EF024C01FF0A6D02D742DA41200010E90
:101650000E6E2E8C1200376A0F5206E10E2A050E0E
:101660000E5C09E30E6A07D00E2A040E0E5C03E33B
:101670000E6A10A60E2A2E8C72681200F7D82D78EA
:10168000F0D82D802E8C72681200376AB8EC02F008
:10169000010E525C12E1050E5A6E8DEC02F00DE364
:1016A000A3EC02F05A2EF9D7B4EC02F0A3EC02F04E
:1016B000020E526E8DEC02F0FDE252501200310427
:1016C00033EC00F0056E00EE13F0040E5A6EBDEF21
:1016D0000BF0310433EC00F0056E00EE17F0040E51
:1016E0005A6EC4EC0BF0310433EC00F0056E00EEE2
:1016F00013F0040E5A6E315209E1136A146A156A26
:10170000166A176A186A196A1A6A1200C4EF0BF08F
:1017100023EC00F0056E00EE1BF0040E5A6E120072
:10172000276A286A296A2A6A2B6AF2DF2DD8EE52C4
:10173000F4DF2AD8EE52020E5A6E26D80D0E0F5C38
:1017400003E3050E5A6E20D82F9425BE2F84259EC4
:1017500088D812008BD82FB4258EDADF0ED8EE523F
:10176000DCDF0BD8EE52020E5A6E07D80D0E0F5C5E
:1017700003E3050E5A6E01D81200EE50066E52D8E1
:10178000052A5A2EFAD7120062D8EE6E052A5A2E72
:10179000FBD71200010E526E2D922E8C72685BEFF9
:1017A00003F0056A0A0E5A6E00EE09F006D8220E02
:1017B000056E0A0E5A6E00EEB7F049D8EE6E052A95
:1017C0005A2EFBD7FE0E056E42D82C6E1200056A0B
:1017D0000A0E5A6E00EE09F006D8220E056E0A0EA9
:1017E0005A6E00EEB7F0EECF06F01CD8052A5A2E3E
:1017F000FAD7FE0E056E2CC006F014D81200000EAB
:10180000F86E7F0EF76E000EF66EF29E2F885A6A03
:10181000056A0900F550066E05D8052A5A2EF9D733
:1018200000EF00F0A6B2FED70550A96E0650A86ED4
:10183000A69EA69CA684F29EF2BEFDD7550EA76E6C
:10184000AA0EA76EA6822FA8F28EA6941200A6B2A8
:10185000FED70550A96EA69EA69CA680A850066E2F
:10186000120025502DB82650326E12002DB831C00E
:1018700026F02DA831C025F0120011521CE0010EF7
:10188000115C10E0020E115C0DE0030E115C37E0FC
:10189000040E115C37E0050E115C37E0060E115C9A
:1018A00037E01200A6EC0CF0A1EC02F0A6EC0CF074
:1018B000A1EC02F012000BD8440E926FBB0E916F98
:1018C0000AD8470E926FAE0E916F6BEF0CF0200EA0
:1018D000926F000E916F8290925104D8915102D86C
:1018E00082801200386E080E5A6E3836D8A0829464
:1018F000D8B08284829282825A2EF7D71200240EA8
:10190000386E08D02C0E386E05D0A40E386E02D07A
:10191000040E386E829282908294829A010E906FA9
:101920000AD8906B08D8906B06D838C090F003D8CE
:10193000828082901200080E5A6E9037D8B082844E
:101940008282829282945A2EF8D712005EC093F05F
:101950005FC094F060C095F061C096F0115211E044
:10196000010E115C29E0020E115C23E04FD0120041
:1019700062C093F063C094F064C095F065C096F0C7
:10198000EDD7A5DF93C091F094C092F0929F928D15
:10199000A2DF933794379537963793379437953737
:1019A000963795C091F096C092F0929F928D6BEF12
:1019B0000CF03B6A3B8001D03B6A93C03AF013D8ED
:1019C00094C03AF010D895C03AF00DD896C03AF0CD
:1019D0000AD83BC03AF007D882800000000082900D
:1019E000000000001200080E5A6E3A32D8A004D04F
:1019F00082840000000001D08294000000008282F6
:101A00000000000082925A2EF0D71200040E906F50
:101A100092DF96C090F08FDF95C090F08CDF94C07D
:101A200090F089DF93C090F086DF82808290120070
:101A300083845BEC03F08DEC02F0FDE2376A010E6B
:101A4000976F2BD837BE0AD037507C0B14E0972BFA
:101A50001B0E975D02E1010E976F0BD037C05DF052
:101A60005D6C5D50FC0B07E09707972902E11A0EA9
:101A7000976F13D8376A8DEC02F0E4E3B8EC02F00C
:101A8000CFEC03F0010E365C03E176D900EF00F0F5
:101A9000040E365CF0E1DEEF0AF0000EF86E340E54
:101AA000F76E7C0EF66E73EC03F0E86A63EC03F0FD
:101AB000010E975D0DE1000EF86E340EF76E8E0E7E
:101AC000F66E76EC03F010A054D910B04FD9120086
:101AD000020E975D0DE1000EF86E340EF76E9E0E4D
:101AE000F66E76EC03F010A444D910B43FD912007E
:101AF000030E975D0DE1000EF86E340EF76EAE0E1C
:101B0000F66E76EC03F010A234D910B22FD9120081
:101B1000040E975D0DE1000EF86E340EF76EBE0EEA
:101B2000F66E76EC03F010A624D910B61FD9120079
:101B3000050E975D0DE1000EF86E340EF76ECE0EB9
:101B4000F66E76EC03F010A814D910B80FD9120075
:101B5000060E975D0DE1000EF86E340EF76EDE0E88
:101B6000F66E76EC03F010AA04D910BAFFD8120072
:101B7000070E975D0DE1000EF86E340EF76EEE0E57
:101B8000F66E76EC03F02FA4F4D82FB4EFD8120041
:101B9000080E975D0DE1000EF86E340EF76EFE0E26
:101BA000F66E76EC03F010ACE4D810BCDFD812006F
:101BB000090E975D0DE1000EF86E350EF76E0E0EF4
:101BC000F66E76EC03F010AED4D810BECFD812006B
:101BD0000A0E975D09E1000EF86E350EF76E1E0EC7
:101BE000F66E76EC03F012000B0E975D09E1000E25
:101BF000F86E350EF76E300EF66E76EC03F01200CE
:101C00000C0E975D09E1000EF86E350EF76E420E70
:101C1000F66E76EC03F012000D0E975D09E1000EF2
:101C2000F86E350EF76E540EF66E76EC03F0120079
:101C30000E0E975D09E1000EF86E350EF76E660E1A
:101C4000F66E76EC03F012000F0E975D09E1000EC0
:101C5000F86E350EF76E780EF66E76EC03F0120025
:101C6000100E975D09E1000EF86E350EF76E880EC6
:101C7000F66E76EC03F01200110E975D0AE1000E8D
:101C8000F86E350EF76E980EF66E76EC03F048EFB0
:101C900014F0120E975D09E1000EF86E350EF76E26
:101CA000A80EF66E76EC03F01200130E975D09E1B4
:101CB000000EF86E350EF76EBA0EF66E76EC03F087
:101CC0001200140E975D09E1000EF86E350EF76EE6
:101CD000CC0EF66E76EC03F01200150E975D09E15E
:101CE000000EF86E350EF76EDE0EF66E76EC03F033
:101CF0001200160E975D09E1000EF86E350EF76EB4
:101D0000F00EF66E76EC03F01200170E975D09E107
:101D1000000EF86E360EF76E020EF66E76EC03F0DD
:101D20001200180E975D09E1000EF86E360EF76E80
:101D3000140EF66E76EC03F01200190E975D09E1B1
:101D4000000EF86E360EF76E260EF66E76EC03F089
:101D500012001A0E975D09E1000EF86E360EF76E4E
:101D6000380EF66E76EC03F012001200310EE8EF3A
:101D700002F0300EE8EF02F08DEC02F0FDE25BECD9
:101D800003F0010E975D01E14AD3020E975D01E178
:101D9000EAD2030E975D01E109D3040E975D01E1DC
:101DA000C3D2050E975D01E1A0D2060E975D01E159
:101DB00057D3070E975D01E133D2080E975D01E11D
:101DC00075D2090E975D01E152D20A0E975D01E1CD
:101DD00062D10B0E975D03E1010E316E50D00C0EF7
:101DE000975D03E1020E316E4AD00D0E975D03E15F
:101DF000030E316E44D00E0E975D03E1040E316E7A
:101E00003ED00F0E975D03E1050E316E38D0100EF7
:101E1000975D03E1060E316E32D0110E975D02E13F
:101E2000C0EF13F0120E975D01E13BD3130E975DE7
:101E300002E16BEF15F0140E975D02E15BEF14F019
:101E4000150E975D02E1F6EF14F0160E975D02E1B4
:101E5000A6EF14F0170E975D02E11FEF16F0180EB3
:101E6000975D02E182EF17F0190E975D02E16BEFCB
:101E700016F01A0E975D02E107EF17F0120031C05D
:101E800025F02D98376A73EC0BF02F8213C09EF06B
:101E900014C09FF015C0A0F016C0A1F05BEC03F0D9
:101EA000000EF86E360EF76EAA0EF66E73EC03F0A7
:101EB000000E986FEAD8000EF86E200EF76E860EB0
:101EC000F66E76EC03F09EC01BF09FC01CF0A0C025
:101ED0001DF0A1C01EF0E6EC03F049EC04F0E86A46
:101EE00063EC03F09EC042F09FC043F0A0C044F0FA
:101EF000A1C045F0B5EC06F01BEC07F00A0E8A6FA6
:101F0000060E8B6F98C08CF0E5EC06F0375201E1BD
:101F10007ED0996B9A6B9B6B9C6B37BE3AD0985373
:101F200008E19E2BD8B49F2BD8B4A02BD8B4A12BFA
:101F30006CD0020E985D0BE1640E996F99519E274B
:101F40009A519F239B51A0239C51A1235ED0040E44
:101F5000985D0DE1100E996F270E9A6F99519E278B
:101F60009A519F239B51A0239C51A1234ED0060E32
:101F7000985D0FE1400E996F420E9A6F0F0E9B6FA6
:101F800099519E279A519F239B51A0239C51A12395
:101F90003CD098530BE19E079E2907E19F079F299C
:101FA00004E1A007A02901E1A1072FD0020E985D4E
:101FB0000BE1640E996F99519E5F9A519F5B9B5103
:101FC000A05B9C51A15B21D0040E985D0DE1100E29
:101FD000996F270E9A6F99519E5F9A519F5B9B5103
:101FE000A05B9C51A15B11D0060E985D0EE1400EE6
:101FF000996F420E9A6F0F0E9B6F99519E5F9A5187
:102000009F5B9B51A05B9C51A15B376A5CD78DECB9
:1020100002F001E27BD7B8EC02F0CFEC03F0010E46
:10202000365C07E1982B982B080E985D01E1986BC0
:102030001BD0020E365C07E19807980798AF02D0D4
:10204000060E986F08D0030E365C01E111D0040E25
:10205000365C01E10ED019D8000EF86E200EF76E36
:10206000860EF66E76EC03F08DEC02F0FDE22BD7D7
:1020700012009EC013F09FC014F0A0C015F0A1C0C4
:1020800016F05FEF0BF04D487A00E86A63EC03F05E
:102090000D0E67EF03F02D982F8209C09EF00AC045
:1020A0009FF00BC0A0F00CC0A1F00DC0A2F05BEC43
:1020B00003F0000EF86E360EF76EAA0EF66E73EC95
:1020C00003F0050E986FE6EC03F049EC04F0DDDF59
:1020D000E86A63EC03F098C05AF000EE0DF0ED50A2
:1020E0006CEC03F05A2EFBD7375261E037BE29D093
:1020F000050E985D09E1092AD8B40A2AD8B40B2A3A
:10210000D8B40C2AD8B40D2A040E985D07E10A2A27
:10211000D8B40B2AD8B40C2AD8B40D2A030E985D73
:1021200005E10B2AD8B40C2AD8B40D2A020E985D0A
:1021300003E10C2AD8B40D2A010E985D01E10D2AA5
:1021400034D0050E985D0DE1090609280AE10A065A
:102150000A2807E10B060B2804E10C060C2801E114
:102160000D06040E985D0AE10A060A2807E10B062F
:102170000B2804E10C060C2801E10D06030E985D06
:1021800007E10B060B2804E10C060C2801E10D0603
:10219000020E985D06E10C060C28D8B40D06D8B4E2
:1021A0000C52010E985D01E10D06376A8CD78DEC5B
:1021B00002F09AE3B8EC02F0CFEC03F0010E365CCB
:1021C00006E19807985302E1050E986F12D0020EAF
:1021D000365C07E1982B060E985D02E1010E986FC0
:1021E00008D0030E365C01E108D0040E365C01E134
:1021F0000FD08DEC02F0FDE266D79EC009F09FC0C3
:102200000AF0A0C00BF0A1C00CF0A2C00DF01200AB
:10221000000E056E00EE09F0050E5A6EBDEF0BF0D4
:10222000000EF86E360EF76E500EF66E73EC03F07D
:10223000000EF86E370EF76E040EF66E73EC03F0B8
:102240008DEC02F0FDE3CFEC03F0010E365C0EE006
:10225000020E365C0BE0030E365C02E12F8404D0E4
:10226000040E365C03E12F94AAEC0BF01200000E72
:10227000F86E370EF76E920EF66E73EC03F0BAD866
:102280008DEC02F0FDE3CFEC03F0010E365C0DE0C7
:10229000020E365C0AE0030E365C02E1388E04D092
:1022A000040E365C02E1389EB4D01200000EF86EC7
:1022B000370EF76E800EF66E73EC03F09BD88DEC44
:1022C00002F0FDE3CFEC03F0010E365C0DE0020EF0
:1022D000365C0AE0030E365C02E1388C04D0040E52
:1022E000365C02E1389C95D01200000EF86E360E76
:1022F000F76EBC0EF66E73EC03F07CD88DEC02F03A
:10230000FDE3CFEC03F0010E365C0DE0020E365C0F
:102310000AE0030E365C02E1388804D0040E365C15
:1023200002E1389876D01200000EF86E360EF76E85
:10233000980EF66E73EC03F05DD88DEC02F0FDE3C1
:10234000CFEC03F0010E365C0DE0020E365C0AE0C5
:10235000030E365C02E1388604D0040E365C01E1DF
:10236000389657D01200000EF86E360EF76E620ED9
:10237000F66E73EC03F03ED88DEC02F0FDE3B8ECA2
:1023800002F0CFEC03F0010E365C0FE0020E365C7B
:102390000CE0030E365C03E13884389205D0040E5D
:1023A000365C02E13894389234D01200000EF86E98
:1023B000360EF76E740EF66E73EC03F01BD88DECD0
:1023C00002F0FDE3B8EC02F0CFEC03F0010E365C56
:1023D00010E0020E365C0DE0030E365C04E138823C
:1023E0003894838405D0040E365C03E13892389427
:1023F00010D01200070E056E27EC0CF006C038F066
:10240000000EF86E360EF76E500EF66E73EC03F09B
:10241000120038C006F0070E056E12EF0CF0000E29
:10242000F86E360EF76E860EF66E73EC03F0E2DF92
:102430008DEC02F0FDE3B8EC02F0CFEC03F0010EFE
:10244000365C0DE0020E365C0AE0030E365C02E1FB
:10245000388004D0040E365C02E13890DAD71200DE
:10246000000EF86E360EF76ECE0EF66E73EC03F0BD
:10247000C1DF8DEC02F0FDE3B8EC02F0CFEC03F02D
:10248000010E365C0DE0020E365C0AE0030E365C8F
:1024900002E1388A04D0040E365C02E1389AB9D7DA
:1024A0001200000EF86E360EF76EE00EF66E73EC4C
:1024B00003F0000EF86E360EF76EF20EF66E73EC49
:1024C00003F08DEC02F0FDE3CFEC03F0040E365C7C
:1024D0000DE0010E365C06E1276A286A296A2A6A3D
:1024E0002B6A4CD18DEC02F0FDE2EBD78DEC02F0C3
:1024F000FDE22D98376A27C09EF028C09FF029C0C2
:10250000A0F02AC0A1F02BC0A2F01B509E271C50A7
:102510009F231D50A0231E50A1231F50A2235BEC1C
:1025200003F0000EF86E360EF76EAA0EF66E73EC20
:1025300003F0000E986FA9DD000EF86E200EF76E06
:10254000860EF66E76EC03F0E86A63EC03F09EC04C
:1025500042F09FC043F0A0C044F0A1C045F0A2C02B
:1025600046F0B5EC06F01BEC07F00B0E8A6F060E7A
:102570008B6F98C08CF0E5EC06F0375201E1B8D0D3
:10258000996B9A6B9B6B9C6B9D6B37BE56D0985327
:102590000AE19E2BD8B49F2BD8B4A02BD8B4A12B82
:1025A000D8B4A22BA3D0020E985D0DE1640E996FF2
:1025B00099519E279A519F239B51A0239C51A1235F
:1025C0009D51A22393D0040E985D0FE1100E996FD8
:1025D000270E9A6F99519E279A519F239B51A023B2
:1025E0009C51A1239D51A22381D0060E985D11E13B
:1025F000400E996F420E9A6F0F0E9B6F99519E2756
:102600009A519F239B51A0239C51A1239D51A2230A
:102610006DD0080E985D11E1E10E9A6FF50E9B6F7B
:10262000050E9C6F99519E279A519F239B51A02381
:102630009C51A1239D51A22359D098530EE19E078E
:102640009E290AE19F079F2907E1A007A02904E12D
:10265000A107A12901E1A20749D0020E985D0DE171
:10266000640E996F99519E5F9A519F5B9B51A05B3D
:102670009C51A15B9D51A25B39D0040E985D0FE186
:10268000100E996F270E9A6F99519E5F9A519F5B1A
:102690009B51A05B9C51A15B9D51A25B27D0060E74
:1026A000985D11E1400E996F420E9A6F0F0E9B6F6D
:1026B00099519E5F9A519F5B9B51A05B9C51A15B7E
:1026C0009D51A25B13D0080E985D10E1E10E9A6F48
:1026D000F50E9B6F050E9C6F99519E5F9A519F5B03
:1026E0009B51A05B9C51A15B9D51A25B376A2CD78B
:1026F0008DEC02F001E241D7B8EC02F0CFEC03F030
:10270000010E365C07E1982B982B0A0E985D01E1CB
:10271000986B1BD0020E365C07E19807980798AFBC
:1027200002D0080E986F08D0030E365C01E111D07C
:10273000040E365C01E10ED0A8DC000EF86E200E0F
:10274000F76E860EF66E76EC03F08DEC02F0FDE28D
:10275000FBD612001B509E5F1C509F5B1D50A05B60
:102760001E50A15B1F50A25B9EC027F09FC028F0A7
:10277000A0C029F0A1C02AF0A2C02BF0AAEF0BF054
:102780008DEC02F0FDE2000EF86E360EF76EAA0E2A
:10279000F66E73EC03F02AD88DEC02F0FDE28DECBE
:1027A00002F0FDE3B8EC02F0CFEC03F0010E365C72
:1027B00006E1112A070E115C01E1116AE1D7020E50
:1027C000365C06E11106112802E1060E116ED8D71B
:1027D000030E365C01E109D0040E365C06E1080EFA
:1027E000056E11C006F012EF0CF01200115209E153
:1027F000000EF86E340EF76E0C0EF66E73EC03F0EE
:1028000047D0010E115C09E1000EF86E340EF76E30
:102810001C0EF66E73EC03F03BD0020E115C09E166
:10282000000EF86E340EF76E2C0EF66E73EC03F09D
:102830002FD0030E115C09E1000EF86E340EF76E16
:102840003C0EF66E73EC03F023D0040E115C09E12C
:10285000000EF86E340EF76E4C0EF66E73EC03F04D
:1028600017D0050E115C09E1000EF86E340EF76EFC
:102870005C0EF66E73EC03F00BD0060E115C08E1F3
:10288000000EF86E340EF76E6C0EF66E73EC03F0FD
:10289000426A436A446A456A466A11C042F0B5EC2E
:1028A00006F01BEC07F0020E8A6F000E8B6F000E15
:1028B0008C6FE5EF06F0376A000EF86E370EF76E94
:1028C000160EF66E73EC03F0000EF86E380EF76E0F
:1028D000280EF66E73EC03F04DEC04F0C0C042F02D
:1028E000B5EC06F01BEC07F0030E8A6F000E8B6F41
:1028F000000E8C6FE5EC06F065EC03F021EC18F0AF
:1029000015EC19F046EC19F08DEC02F00BE3B8EC85
:1029100002F0CFEC03F0040E365C01E11200010E70
:10292000365C11E03752F0E037BE05D037A8ECD75F
:10293000C02B376AC9D7376C37A803D0C007376AAE
:10294000C3D7376CE1D7E7EC0BF01200000EF86E3E
:10295000370EF76E160EF66E73EC03F0000EF86E7F
:10296000380EF76E1A0EF66E73EC03F04DEC04F0B1
:1029700012C042F0050E4A6E01EC06F06CEC04F059
:10298000B5EC06F01BEC07F0040E8A6F000E8B6F9F
:10299000000E8C6FE5EC06F0000EF86E380EF76E48
:1029A000240EF66E76EC03F08DEC02F00BE3B8EC3F
:1029B00002F0CFEC03F0040E365C01E11200010ED0
:1029C000365C11E03752F0E037BE05D037A8ECD7BF
:1029D000122A376AC3D7376C37A803D01206376A72
:1029E000BDD7376CE1D7E7EC0BF01200000EF86EA4
:1029F000370EF76E160EF66E73EC03F02D84BBECFB
:102A000003F0000EF86E370EF76EA40EF66E73EC40
:102A100003F0436A446A456A466ABFC042F0B5ECB7
:102A200006F038506CEC03F0300EE8EC02F0000ECB
:102A3000F86E370EF76EAA0EF66E76EC03F08DEC9C
:102A400002F00BE3B8EC02F0CFEC03F0040E365CBE
:102A500001E11200010E365C11E03752F0E037BEA2
:102A600005D037A8ECD7BF2B376AC8D7376C37A843
:102A700003D0BF07376AC2D7376CE1D7E7EC0BF05A
:102A80001200000E63EC03F0BA516CEC03F0B95184
:102A90006CEC03F0B8516CEC03F0B7516CEC03F044
:102AA00065EC03F0400E63EC03F0BE516CEC03F0F8
:102AB000BD516CEC03F0BC516CEC03F0BB516CEC01
:102AC00003F065EC03F097EF02F08E516CEC03F02D
:102AD0008D516CEF03F0000EF86E370EF76E160E88
:102AE000F66E73EC03F0000EF86E370EF76E280EDC
:102AF000F66E73EC03F06AEC09F0E7DFA1EC02F08C
:102B00008DEC02F0F0E3B8EC02F0CFEC03F0040E31
:102B1000365C01E11200010E365C01E0E4D78DEC79
:102B200002F0FDE28DC000F18EC001F1000EF86EE2
:102B3000370EF76E300EF66E73EC03F06AEC09F0A8
:102B4000C4DFA1EC02F08DEC02F0F0E3B8EC02F08F
:102B5000CFEC03F0040E365C01E11200010E365C8E
:102B600001E0E4D78DEC02F0FDE28DC002F18EC0F1
:102B700003F14DEC04F000C142F001C143F002C189
:102B80004AF003C14BF042504A5E43504B5A445006
:102B90004C5A45504D5A46504E5A4FEC04F0A00E38
:102BA000426EF00E436E190E446E6AEC06F038C0A9
:102BB000B7F039C0B8F03AC0B9F03BC0BAF04DEC4C
:102BC00004F000C142F001C143F0B7C04AF0B8C000
:102BD0004BF0B9C04CF0BAC04DF001EC06F0381E15
:102BE000391E3A1E3B1E3C1E382AD8B4392AD8B4A6
:102BF0003A2AD8B43B2AD8B43C2A38C0BBF039C0F2
:102C0000BCF03AC0BDF03BC0BEF0000EF86E370E0F
:102C1000F76E380EF66E73EC03F08DEC02F0FDE308
:102C2000CFEC03F0040E365C01E11200010E365CBD
:102C300001E0F3D75BEC03F024DFE7EF0BF0000ECD
:102C4000F86E370EF76E4A0EF66E73EC03F0000E58
:102C5000F86E370EF76E160EF66E73EC03F08DEC11
:102C600002F0FDE3B8EC02F0CFEC03F0040E365CAA
:102C700001E11200CFEC03F0010E365C01E0DFD77A
:102C80005BEC03F0000EF86E370EF76E4A0EF66E30
:102C900073EC03F0F29E2F885C6A056A400E63ECC9
:102CA00003F005506CEC03F027EC0CF078EC02F02C
:102CB000A5EC02F0052A5C2EF1D7000EF86E370E57
:102CC000F76E5C0EF66E73EC03F097EC02F08DEC91
:102CD00002F0FDE21200000EF86E370EF76EAE0E37
:102CE000F66E73EC03F0000EF86E370EF76E160EEC
:102CF000F66E73EC03F08DEC02F0FDE3B8EC02F03D
:102D0000CFEC03F0040E365C01E11200CFEC03F0CF
:102D1000010E365C01E0DFD78DEC02F0FDE2000E23
:102D2000F86E370EF76EC00EF66E73EC03F0000E01
:102D3000F86E370EF76ED20EF66E73EC03F08DEC74
:102D400002F0FDE3B8EC02F0CFEC03F0010E365CCC
:102D500015E0CFEC03F0020E365C17E0CFEC03F089
:102D6000030E365C19E0CFEC03F0040E365C000E67
:102D7000F86E7E0EF76E000EF66E14D0000EF86E32
:102D80007B0EF76E000EF66E0DD0000EF86E7C0E08
:102D9000F76E000EF66E06D0000EF86E7D0EF76E22
:102DA000000EF66EF29E2F885C6A056A03EE00F054
:102DB00027EC0CF0EE6E052A5C2EFAD703EE00F03D
:102DC0000ED8000EF86E370EF76E5C0EF66E73ECD2
:102DD00003F09AEC02F08DEC02F0FDE21200200EFE
:102DE000F36EF80EF616080EEECFF5FF0C00090094
:102DF000E82EFAD70A00840EA66E550EA76EAA0E0C
:102E0000A76EA68200000900F32EEBD71200838480
:102E1000000EF86E370EF76EF60EF66E73EC03F0DA
:102E2000000EF86E370EF76E160EF66E73EC03F0AA
:102E30008DEC02F0FDE28DEC02F0FDE3B8EC02F067
:102E4000CFEC03F0040E365C01E11200CFEC03F08E
:102E5000010E365C01E0DBD78DEC02F0FDE2000EE6
:102E6000F86E370EF76EC00EF66E73EC03F0000EC0
:102E7000F86E370EF76ED20EF66E73EC03F08DEC33
:102E800002F0FDE3B8EC02F0CFEC03F0010E365C8B
:102E900015E0CFEC03F0020E365C17E0CFEC03F048
:102EA000030E365C19E0CFEC03F0040E365C000E26
:102EB000F86E7E0EF76E000EF66E14D0000EF86EF1
:102EC0007B0EF76E000EF66E0DD0000EF86E7C0EC7
:102ED000F76E000EF66E06D0000EF86E7D0EF76EE1
:102EE000000EF66E05EC0CF0000EF86E370EF76E65
:102EF0005C0EF66E73EC03F09AEC02F08DEC02F0CF
:102F0000FDE21200000EF86E370EF76E6E0EF66ED2
:102F100073EC03F0000EF86E370EF76E160EF66EB9
:102F200073EC03F08DEC02F0FDE3B8EC02F0CFECB3
:102F300003F0040E365C01E11200CFEC03F0010E49
:102F4000365C01E0DFD75BEC03F0000EF86E370E65
:102F5000F76E6E0EF66E73EC03F0F29E2F885D6ACC
:102F6000056A03EE00F0400E63EC03F005506CECD4
:102F700003F065EC03F074EC02F0EE6E066E6CECA0
:102F800003F0052A5D2EEFD7650E065C16E05BECBC
:102F900003F0000EF86E380EF76EB00EF66E73EC9E
:102FA00003F006506CEC03F0000EF86E380EF76E6E
:102FB000BE0EF66E73EC03F015D0F29E2F885D6A9C
:102FC000056A03EE00F0EECF06F012EC0CF0052AD5
:102FD0005D2EF9D7000EF86E370EF76E5C0EF66EAA
:102FE00073EC03F097EC02F08DEC02F0FDE21200BE
:102FF00015EE00F0E1CFC3F0E2CFC4F0E1CFC1F0B5
:10300000E2CFC2F01D0EAF6EAC94AC8AAB88AB8E33
:103010001200C3C0E1FFC4C0E2FFC151E15C02E1A4
:10302000D89012002E98E650C56FF10EE15C02E1D7
:1030300015EE00F0E1CFC3F0E2CFC4F0C551D88067
:103040001200080E5B6E696A6A6A6B6A6C6A72ECDF
:1030500009F08D5169268E516A2270EC09F08D516C
:103060006B268E516C225B2EF2D712008DEC02F093
:10307000FDE24BEC04F0838083825BEC03F04DECCB
:1030800004F0DFDF6A506C5C02E169506B5C05E3C1
:10309000270E436E0F0E426E3FD069C042F06AC0E9
:1030A00043F0446A456A466A6B5042266C5043229C
:1030B000000E4B6E640E4A6E4C6A4D6A4E6A4F6A41
:1030C000506A01EC06F038C042F039C043F03AC013
:1030D00044F03BC045F03CC046F038C079F039C000
:1030E0007AF069C04AF06AC04BF04C6A4D6A4E6A89
:1030F0006B504A5E6C504B5A6AEC06F038C042F096
:1031000039C043F03AC044F03BC045F03CC046F003
:1031100038C0A3F039C0A4F0B5EC06F01BEC07F002
:10312000040E8A6F020E8B6F8C6B000EF86E360EDB
:10313000F76E4A0EF66E73EC03F0E5EC06F0A5ECC4
:1031400002F073D865EC03F0A1D84DEC04F0A3C0F5
:1031500042F0A4C043F0640E4A6E4A50425E4B50A7
:10316000435A4C50445A4D50455A4E50465A58ECCA
:1031700004F0640E4A6E01EC06F06CEC04F058ECBE
:1031800004F0710E4A6E020E4B6E6AEC06F06CECA7
:1031900004F058EC04F0020E4A6E6AEC06F0100ED1
:1031A000385C05E3100EA56FA66BA76B0BD038C07B
:1031B000A5F042C0A6F0100E426EA551425CA76F6A
:1031C000A667A707400E63EC03F0A56702EC19F0B1
:1031D000A6670AEC19F0A7670DEC19F08DEC02F068
:1031E00002E281B24CD7B8EC02F02D948392839026
:1031F00049EC04F081A2FED78DEC02F0FBE2A1ECD9
:1032000002F01200A5C05AF0010EE8EC02F05A2EAE
:10321000FBD71200000EE8EF02F0A7C05AF0060E2E
:10322000E8EC02F05A2EFBD712004DEC04F069C016
:1032300042F06AC043F0040E4B6EE20E4A6E01EC9F
:1032400006F04EEC04F06CEC04F0080E4A6E6AECEA
:1032500006F039C042F03AC043F03BC044F03CC0F5
:1032600045F0C0C04AF001EC06F06CEC04F077ECDD
:1032700004F001EC06F04EEC04F06CEC04F0C30E2C
:103280004B6E500E4A6E6AEC06F012006CEC04F0C5
:10329000080E8A6F830E8C6F4D6A4E6A0F0E4C6E4D
:1032A000420E4B6E3F0E4A6E4E50465C0BE14D5047
:1032B000455C08E14C50445C05E14B50435C02E145
:1032C0004A50425C04E2820E8C6F060E8A6F4D6A91
:1032D0004E6A010E4C6E860E4B6E9F0E4A6E4E501D
:1032E000465C0BE14D50455C08E14C50445C05E107
:1032F0004B50435C02E14A50425C04E2810E8C6F09
:10330000050E8A6FB5EC06F01BEC07F0030E8B6F11
:10331000E5EC06F0570EE8EC02F0120010AC1200DB
:10332000800E78EC02F00F5078EF02F010AC120033
:10333000810E78EC02F0315078EF02F0006ED8CFB9
:1033400001F0E0CF02F0EACF04F0E9CF03F0C2C011
:10335000EAFFC1C0E9FF9EAA0ED0AE50ABA204D0D6
:10336000AE50AB98AB88F7D7EE6EF10EE95C02E198
:1033700005EE00F0F0D7EACFC2F0E9CFC1F0F2A439
:1033800007D0F29466C0D6FF2DB480782DA4809823
:10339000F2A207D0D02B81A602D0370601D0372A5F
:1033A000F2929EA00BD09E9053665306546654062C
:1033B00057665706000ECE6EA60ECF6EA1B8A19826
:1033C0009EA204D09E92565201E0560604C0EAFF27
:1033D00003C0E9FF02C0E0FF005001C0D8FF1000A9
:1033E000006ED8CF01F0E0CF02F002C0E0FF005045
:1033F00001C0D8FF100040286329444C344A414C96
:103400002056613A313520000C2E0000004144392D
:103410003833332F414439383334200000414439A4
:103420003835302F3531202020202000004144390C
:1034300038353120504C4C2A362020000041443988
:1034400039353120504C4C2A342020000041443979
:1034500039353120504C4C2A352020000041443968
:1034600039353120504C4C2A32302000004144394B
:10347000393531206F2E20504C4C2000405345549C
:103480002020202020204162627275636800303164
:1034900020532D4D6574657220202020200030328D
:1034A000204C69636874206175746F20200030338C
:1034B000204C69636874207065726D2E2000303472
:1034C000204672712031487A20202020200030359B
:1034D000204B657965722020202020202000303686
:1034E000205458205A46207065726D2E20003037C7
:1034F0002056464F3D52582D5A4620202000303845
:103500002042616E642F4D6F6465202020003039A9
:103510002056464F783420492F516D69780031305C
:10352000204444532D436F6E7374202020200000EC
:103530003131205A462043572020202020202020AF
:1035400000003132205A462043572052657665727A
:10355000732000003133205A46204C534220202053
:103560002020202000003134205A4620555342208C
:1035700020202020202000003135205A46204162A2
:103580006C2E203630306B003136205A4620416296
:103590006C2E373630306B00313720444453205482
:1035A00079706520202000003138204C4344736836
:1035B000696674202B20525800003139204B616C11
:1035C0002E2020532D4D6574657200003230204B43
:1035D000616C2E204C65697374756E670000323122
:1035E000204D6974686F6572746F6E202020000032
:1035F00032322054582068616E672074696D6520EE
:103600000000323320456570722E205049432D3E14
:1036100050430000323420456570722E2050432DF7
:103620003E504943000032352045657072202D3EE2
:1036300020466C6173680000323620466C61736806
:10364000202D3E20456570720000005357563D0006
:1036500040582020205820202065696E2020617568
:103660007300004C696368746175746F6D6174698F
:103670006B202000004C69636874202020202020EB
:1036800020202020200000532D4D657465722020DD
:103690002020202020202000003120487A20417561
:1036A000666C6F6573756E672000403C2020203E7D
:1036B0002020202058202020206F6B00004B6579AF
:1036C000657220202020202020202020200000546F
:1036D00058205A46207065726D616E656E742000C8
:1036E00000446973706C617973686966743D302059
:1036F0002000406A6120202020202020207765695A
:10370000746572000056464F203D20525866727113
:10371000202D205A4600404F4B20202020202020E2
:103720004162627275636800005330203D200000E2
:10373000005339203D2000000053706569636865BF
:10374000726E3F2020202020200000504943202D71
:103750002D2D3E20504320205458200040466572B5
:103760007469672120202020202020202000005084
:1037700043202D2D2D3E205049432020525820001B
:103780000042616E642F4D6F646520616B746976D1
:1037900020000056464F783420492F51204D69783B
:1037A00065722000004D543D200020487A000045FD
:1037B0006570726F6D202D2D3E20466C6173680020
:1037C000005370656963686572706C61747A20205B
:1037D00020004031202020203220202020332020B3
:1037E00020203400402020202020202020202020C5
:1037F00020202020200000466C617368202D2D3E83
:1038000020456570726F6D0000456570722E6175A0
:1038100066667269736368656E0000545868616E0D
:10382000673D2000206D53000066616B3D000D4D2B
:10383000487A00000D43572000000D4357720000E6
:103840000D4C534200000D55534200000D413036DF
:1038500000000D41373600004042616E64776563B9
:103860006873656C2020202020000820566F6C743F
:1038700000004057704D3A20000000446174656EAE
:1038800020696D2042756666657220000055726C75
:103890006164756E672020202020202020000055C4
:1038A000726C6164756E67206265656E6465740034
:1038B0000041626272756368202121210000404648
:1038C000616C736368657320466F726D617421006B
:1038D000403120412F42205354455020524954201A
:1038E0002000403220413D42204D746F6E20313027
:1038F000306B2000403320423D4120204D656D203B
:1039000053417574200040342053575620205345AE
:1039100054205562617420004035202043572020F8
:103920004C534220555342202000403620435772CA
:103930002020413036204137362020004037204DAE
:10394000657373203136306D2038306D200040387B
:1039500020202036306D2034306D2033306D200033
:10396000403920202032306D2031376D2031356DC7
:103970002000403130202031326D2031306D202048
:10398000366D20004031312020326D20207472319C
:10399000207472322000403132202074723320743F
:1039A00072342074723520000056312E31372020B9
:0A39B0002030352E31322E31340064
:107F00001771C7BC0A010252060120A1070020A177
:107F1000070040420F0060E3160080841E0080844A
:107F20001E00180C00002887F9FF44018096980075
:107F3000809698000000509E1B00903A1C000103A0
:107F400040523600207538000103205C5100205C4F
:107F500051000103F0446B0060566C000103201DCA
:107F60009A00201D9A000104E089D600C0ACD80018
:107F70000104801F1401801F14010104A059410154
:107F800030B94201010490CA7B0190CA7B0101040F
:107F90006029AC01E0D2AF0101040029FC020029F4
:107FA000FC020104E0D79908E0D799080104003FDA
:107FB000AB01003FAB010104000000000000003FE6
:107FC000AB01003FAB010104000000000000003FD6
:107FD000AB01003FAB010104000000000000003FC6
:107FE000AB01003FAB010104000000000000003FB6
:107FF000AB01003FAB01010400000000000001657F
:020000040030CA
:03000100220D0EBF
:02000500018177
:00000001FF
